:100000000C9461010C9489010C9489010C94890170
:100010000C9489010C9489010C9489010C94890138
:100020000C9489010C9489010C9489010C94890128
:100030000C9489010C9489010C9489010C94890118
:100040000C948B230C9489010C947E250C94B02580
:100050000C9489010C9489010C9489010C948901F8
:100060000C9489010C9489013C76657273696F6EFA
:1000700020302E3934393E00467265652052414D9C
:100080003A20004552524F523A200053797320765D
:100090006F6C74733A200053797320766F6C7473AD
:1000A000206368617267696E673A20005379732034
:1000B000766F6C74732069646C653A2000626174B9
:1000C00074506C757350696E204F4E006261747489
:1000D000506C757350696E204F464600637572729E
:1000E000656E745A65726F4F66667365743A005335
:1000F000616D706C652073697A653A20003E00205E
:1001000000200020002000200020002000200020EF
:10011000003C0041444A555354494E472000616415
:100120006A416D70735F4F4E200061646A566F6C58
:1001300074735F4F4E200063656C6C5368756E740A
:10014000335F4F4E200063656C6C5368756E74327C
:100150005F4F4E200063656C6C5368756E74315F41
:100160004F4E200074617267657420416D70733A60
:10017000200074617267657420566F6C74733A2046
:100180000070777250574D3A200049444C45205436
:100190004F54414C20566F6C74733A200049444CC4
:1001A0004520566F6C747320333A200049444C4507
:1001B00020566F6C747320323A200049444C45201D
:1001C000566F6C747320313A2000434841524749BE
:1001D0004E4720544F54414C20566F6C74733A2054
:1001E000004348415247494E4720566F6C74732074
:1001F000333A20004348415247494E4720566F6CDE
:10020000747320323A20004348415247494E4720F8
:10021000566F6C747320313A20004348415247496D
:100220004E472063757272656E7420414D50533A8B
:100230002000544F54414C20766F6C74733A200068
:10024000766F6C747320333A2000766F6C74732071
:10025000323A2000766F6C747320313A2000437577
:100260007272656E7420416D70733A200000000058
:100270000800020100000304070000000000000065
:10028000000102040810204080010204081020012F
:1002900002040810200404040404040404020202FA
:1002A00002020203030303030300000000250028E9
:1002B000002B0000000000240027002A0000572027
:1002C000E02511241FBECFEFD8E0DEBFCDBF15E083
:1002D000A0E0B1E0E4EFF8E502C005900D92A63091
:1002E000B107D9F726E0A6E0B5E001C01D92AC3811
:1002F000B207E1F712E0C2ECD2E004C02297FE019F
:100300000E945E2CCE3BD107C9F70E9424260C9494
:10031000782C0C94000060E084E00E94482581E085
:1003200080939C050895CF93DF9300D000D0CDB784
:10033000DEB79A01AB01BC01882777FD8095982F25
:1003400029833A834B835C830E94F72A29813A816F
:100350004B815C810E94AB2B20E030EC4FE754E4F2
:100360000E945C2A20E030E040E250E40E94F32941
:1003700024EA30E74DE35EE30E945C2A0F900F9081
:100380000F900F90DF91CF9108958091DD059091AE
:10039000DE05A091DF05B091E0058093BA0590934A
:1003A000BB05A093BC05B093BD0580913E01909123
:1003B0003F01A0914001B0914101803D9740A105CE
:1003C000B105F1F460E070E085E00E94872460E010
:1003D00088E00E94482561E087E00E94482561E0AE
:1003E00084E00E94482588EC90E0A0E0B0E0809393
:1003F0003E0190933F01A0934001B09341012EC074
:1004000080919E05882321F061E088E00E944825C4
:1004100080919D05882321F060E087E00E944825B7
:1004200080919C05882321F060E084E00E944825AB
:100430006091C4057091C50585E00E94872480ED18
:1004400097E0A0E0B0E080933E0190933F01A0933D
:100450004001B093410181E08093B90580913A0158
:1004600090913B01A0913C01B0913D014091DD058F
:100470005091DE056091DF057091E005840F951FB6
:10048000A61FB71F8093D5059093D605A093D705D7
:10049000B093D8051092D1051092D2051092D305D1
:1004A0001092D40508958091DD059091DE05A0910C
:1004B000DF05B091E0058093CD059093CE05A09324
:1004C000CF05B093D00561E571E08BEE95E00E9419
:1004D000E22780911501909116018130910519F460
:1004E00065E571E009C0009719F463E571E004C0A7
:1004F000019631F46DE571E08BEE95E00E94E22704
:1005000020911B0130911C0140911D0150911E0151
:1005100060914F0570915005809151059091520561
:100520000E945C2A20E030E048EC52E40E94AB2BB1
:100530000E94C42A4AE050E08BEE95E00E94C62853
:1005400066E671E08BEE95E00E94E2278091B805A7
:10055000882331F068E671E08BEE95E00E94E22797
:1005600062E771E08BEE95E00E94E2278091B8058A
:10057000882309F4CCC040916605509167056091CD
:1005800068057091690522E030E08BEE95E00E94ED
:10059000DE296AE771E08BEE95E00E94E227409148
:1005A000620550916305609164057091650522E0D4
:1005B00030E08BEE95E00E94DE296AE771E08BEE79
:1005C00095E00E94E22740915E0550915F056091A1
:1005D00060057091610522E030E08BEE95E00E94AD
:1005E000DE296CE771E08BEE95E00E94E2274091F6
:1005F000760550917705609178057091790522E034
:1006000030E08BEE95E00E94DE296AE771E08BEE28
:1006100095E00E94E2274091720550917305609128
:1006200074057091750522E030E08BEE95E00E9434
:10063000DE296AE771E08BEE95E00E94E2274091A7
:100640006E0550916F05609170057091710522E003
:1006500030E08BEE95E00E94DE2963E871E08BEEDE
:1006600095E00E94E22780919E05882319F068E5B5
:1006700074E002C062E973E08BEE95E00E94E2272D
:1006800080919D05882319F068E574E002C062E955
:1006900073E08BEE95E00E94E22780919C05882311
:1006A00019F068E574E002C062E973E08BEE95E052
:1006B0000E94E2278091C605882331F068E871E046
:1006C0008BEE95E00E94E2276AE871E08BEE95E000
:1006D0000E94E22740915A0550915B0560915C05AC
:1006E00070915D0522E030E08BEE95E00E94DE29FE
:1006F00060E971E08BEE95E00E94E22740916A0587
:1007000050916B0560916C0570916D0544C04091EE
:10071000860550918705609188057091890522E0D2
:1007200030E08BEE95E00E94DE296AE771E08BEE07
:1007300095E00E94E22740918205509183056091E7
:1007400084057091850522E030E08BEE95E00E94F3
:10075000DE296AE771E08BEE95E00E94E227409186
:100760007E0550917F05609180057091810522E0A2
:1007700030E08BEE95E00E94DE2966E971E08BEEB9
:1007800095E00E94E22740917A0550917B056091A7
:100790007C0570917D0522E030E08BEE95E00E94B3
:1007A000DE296BE971E08BEE95E00E94E227609113
:1007B000C4057091C5054AE050E08BEE95E00E94BB
:1007C000C62861EA71E08BEE95E00E94E2278091F5
:1007D000B805882349F0409156055091570560911E
:1007E00058057091590508C040918A0550918B05B4
:1007F00060918C0570918D0522E030E08BEE95E0E4
:100800000E94DE2968EA71E08BEE95E00E94E22703
:1008100060914F057091500580915105909152055E
:100820000E94C42A4AE050E08BEE95E00E94C62860
:100830006EEA71E08BEE95E00E94E227409117018D
:10084000509118016091190170911A0122E030E075
:100850008BEE95E00E94DE2980E090E0A6ECB2E409
:100860008093170190931801A0931901B0931A0176
:1008700063EB71E08BEE95E00E94E2274091240546
:1008800050912505609126057091270522E030E002
:100890008BEE95E00E94DE2968EB71E08BEE95E02F
:1008A0000E94E22780910A01882319F062E973E02F
:1008B00002C068E574E08BEE95E00E94E2276DEBE4
:1008C00071E08BEE95E00E94E227609153057091F4
:1008D00054054AE050E08BEE95E00E94C62865E49E
:1008E00072E08BEE95E00C9411286091C405709134
:1008F000C50585E00E9487244091DD055091DE0505
:100900006091DF057091E00580913A0190913B0183
:10091000A0913C01B0913D01840F951FA61FB71F08
:100920008093D5059093D605A093D705B093D805AD
:1009300080ED97E0A0E0B0E080933E0190933F010E
:10094000A0934001B093410148535F4F6F4F7F4FD9
:100950004093BA055093BB056093BC057093BD05E9
:100960001092C60508954F925F926F927F928F9278
:100970009F92AF92BF92CF92DF92EF92FF920F932E
:100980001F93CF93DF93CDB7DEB728970FB6F894B8
:10099000DEBF0FBECDBF00919A0510919B058091DF
:1009A000960590919705B8010E94122CCB014FE655
:1009B00052E163E870E40E94930120912405309194
:1009C000250540912605509127050E94F4296D8345
:1009D0007E838F83988760938A0570938B058093BD
:1009E0008C0590938D05C090D105D090D205E090F4
:1009F000D305F090D405C114D104E104F10409F445
:100A000048C06091DD057091DE058091DF05909111
:100A1000E0056C197D098E099F090E94F52A20E0E6
:100A20003AEB4BE55AE40E945C2A2D813E814F81CE
:100A300058850E94AB2B20E030E04AE754E40E9446
:100A4000AB2B20914F0530915005409151055091AD
:100A500052050E94F42960934F05709350058093CE
:100A6000510590935205C0901B01D0901C01E0905D
:100A70001D01F0901E01A70196010E94A72B1816D8
:100A800044F4C0924F05D0925005E0925105F09287
:100A900052058091940590919505B8010E94122C01
:100AA000882777FD8095982F0E94F72A20E030EC68
:100AB0004FE754E40E945C2A2FE632E143E850E419
:100AC0000E94AB2B2AEF39E146E55FE30E945C2AE6
:100AD00020E030E0A9010E94F4296B017C016093C1
:100AE000860570938705809388059093890580918A
:100AF000920590919305B8010E94122C882777FDEA
:100B00008095982F0E94F72A20E030EC4FE754E4BC
:100B10000E945C2A2FE632E143E850E40E94AB2BAE
:100B200021EE3FE641EE5EE30E945C2AA7019601BA
:100B30000E94F32920E030E0A9010E94F4294B0132
:100B40005C01609382057093830580938405909384
:100B500085058091900590919105B8010E94122C15
:100B60003B01A5019401C701B6010E94F4296983E4
:100B70007A838B839C83B301882777FD8095982F98
:100B80000E94F72A20E030EC4FE754E40E945C2AF0
:100B90002FE632E143E850E40E94AB2B2FEF35EE15
:100BA00042E95EE30E945C2A29813A814B815C81A3
:100BB0000E94F32920E030E0A9010E94F4292B01D2
:100BC0003C0160937E0570937F0580938005909330
:100BD00081059B01AC0169817A818B819C810E9496
:100BE000F42969837A838B839C8320911701309148
:100BF00018014091190150911A010E94582A87FF4B
:100C00000CC089819A81AB81BC818093170190933C
:100C10001801A0931901B0931A0180918E0590914B
:100C20008F05B8010E94122C882777FD8095982F98
:100C30000E94F72A20E030EC4FE754E40E945C2A3F
:100C40002FE632E143E850E40E94AB2B27E53FE377
:100C500048E65EE30E945C2A60937A0570937B0508
:100C600080937C0590937D051092970510929605D0
:100C7000109295051092940510929305109292058A
:100C8000109291051092900510928F0510928E058A
:100C9000109399050093980510929B0510929A0560
:100CA0002091B805222309F403C12091B90522231C
:100CB00019F1C0927605D0927705E0927805F0920E
:100CC00079058092720590927305A0927405B09296
:100CD000750540926E0550926F0560927005709296
:100CE000710560936A0570936B0580936C05909312
:100CF0006D051092B905DCC0C0926605D0926705FB
:100D0000E0926805F0926905809262059092630511
:100D1000A0926405B092650540925E0550925F0511
:100D2000609260057092610560935A0570935B054F
:100D300080935C0590935D058D819E81AF81B88520
:100D40008093560590935705A0935805B093590585
:100D5000A5019401C701B6010E94A72B87FD11C010
:100D6000A3019201C701B6010E94A72B87FD09C00C
:100D7000C0929F05D092A005E092A105F092A20535
:100D800021C0A7019601C501B4010E94A72B87FDD0
:100D900011C0A3019201C501B4010E94A72B87FDD8
:100DA00009C080929F059092A005A092A105B092E3
:100DB000A20508C040929F055092A0056092A1052F
:100DC0007092A2052AE037ED43E25DE360913201C3
:100DD0007091330180913401909135010E94F42982
:100DE0009B01AC0160919F057091A0058091A105C8
:100DF0009091A2050E94A72B181604F58091B705C3
:100E00008823E1F08091C4059091C505059797FD71
:100E100005C09093C5058093C40504C01092C50514
:100E20001092C4050E94750480915505882331F005
:100E300062EC71E08BEE95E00E94112820912E016A
:100E400030912F0140913001509131016091560550
:100E50007091570580915805909159050E94F3298A
:100E600029E23CE54FE05EE30E94A72B181604F54B
:100E70008091B7058823E1F08091C4059091C50564
:100E8000059797FD05C09093C5058093C40504C0E0
:100E90001092C5051092C4050E94750480915505F5
:100EA000882331F065ED71E08BEE95E00E9411280A
:100EB0008091DD059091DE05A091DF05B091E00500
:100EC0008093D1059093D205A093D305B093D40518
:100ED00028960FB6F894DEBF0FBECDBFDF91CF913D
:100EE0001F910F91FF90EF90DF90CF90BF90AF9048
:100EF0009F908F907F906F905F904F9008954F924A
:100F00005F926F927F928F929F92AF92BF92CF9299
:100F1000DF92EF92FF920F931F93CF93DF93CDB7A2
:100F2000DEB728970FB6F894DEBF0FBECDBF809115
:100F3000DD059091DE05A091DF05B091E0058D8380
:100F40009E83AF83B8878093C9059093CA05A09309
:100F5000CB05B093CC058091C8058823A9F080907B
:100F6000480190904901A0904A01B0904B01C09077
:100F70009F05D090A005E090A105F090A2058AE021
:100F800097EDA3EABCE314C0809044019090450122
:100F9000A0904601B0904701C0905605D0905705EB
:100FA000E0905805F090590589E29CE5AFE8BDE373
:100FB00089839A83AB83BC83A5019401C701B601E1
:100FC0000E94F3292B013C0120E030E0A9010E949E
:100FD000A72B181624F077FA709477F8709429816B
:100FE0003A814B815C81C301B2010E94A72B87FD2E
:100FF000EAC08091C6050091C4051091C505811114
:101000004BC081E08093C6058D819E81AF81B885FC
:101010008093BE059093BF05A093C005B093C10512
:10102000A5019401C701B6010E94582A87FF03C099
:1010300081E090E002C08FEF9FEF9093C305809313
:10104000C20520E030E040E850E469817A818B817C
:101050009C810E94AB2B9B01AC01C301B2010E9499
:10106000A72B18161CF485E090E002C081E090E008
:10107000909343018093420140914201509143017A
:101080002091C2053091C305429FC001439F900D3E
:10109000529F900D112441C0A5019401C701B601D2
:1010A0000E94582A6090C2057090C30587FF11C046
:1010B0009FEF6916790669F481E090E0909343010F
:1010C000809342019093C3058093C205C8010196A5
:1010D00026C0A5019401C701B6010E94A72B1816CE
:1010E0008CF4A1E06A16710469F470924301609275
:1010F00042018FEF9FEF9093C3058093C205C80113
:1011000001970DC02091420130914301269DC001FD
:10111000279D900D369D900D1124800F911F909367
:10112000C5058093C4058091C4059091C505853B94
:1011300091053CF084EB90E09093C5058093C40545
:1011400006C097FF04C01092C5051092C4056091B7
:10115000C4057091C50585E00E9487244091DD0596
:101160005091DE056091DF057091E00580913A01B4
:1011700090913B01A0913C01B0913D01840F951FDE
:10118000A61FB71F8093D5059093D605A093D705CA
:10119000B093D80580ED97E0A0E0B0E080933E01E9
:1011A00090933F01A0934001B093410148535F4F9A
:1011B0006F4F7F4F4093BA055093BB056093BC05BA
:1011C0007093BD0502C01092C60528960FB6F8941C
:1011D000DEBF0FBECDBFDF91CF911F910F91FF906A
:1011E000EF90DF90CF90BF90AF909F908F907F90C7
:1011F0006F905F904F9008951092C5051092C405AE
:1012000060E070E085E00E9487241092C70510928C
:10121000C8051092C60585E090E090934301809345
:10122000420108958130910589F4662341F061E01F
:1012300088E00E94482581E080939E05089560E043
:1012400088E00E94482510929E05089582309105FD
:1012500089F4662341F060E087E00E94482581E040
:1012600080939D05089561E087E00E9448251092D3
:101270009D050895039749F461110C948B0161E079
:1012800084E00E94482510929C0508950E94FC0865
:1012900060E081E090E00E94120960E082E090E06E
:1012A0000E94120960E083E090E00C941209CF9252
:1012B000DF92EF92FF92CF93DF9300D000D0CDB7B3
:1012C000DEB720915305309154052330310579F173
:1012D00021E02093B70569837A838B839C830E94E6
:1012E0004609C090DD05D090DE05E090DF05F09066
:1012F000E00569817A818B819C81C60ED71EE81E2C
:10130000F91EB701A6014C53564F6F4F7F4F4093C4
:10131000B3055093B4056093B5057093B605C092BC
:10132000A705D092A805E092A905F092AA050F9012
:101330000F900F900F90DF91CF91FF90EF90DF9083
:10134000CF9008954F925F926F927F928F929F926B
:10135000AF92BF92CF92DF92EF92FF92CF93DF9343
:1013600000D000D0CDB7DEB749835A836B837C832E
:1013700081309105A1F4222309F44FC0C090760575
:10138000D0907705E0907805F0907905409072054F
:1013900050907305609074057090750516C082308A
:1013A0009105E1F4222309F449C0C0907205D09060
:1013B0007305E0907405F0907505409076055090A7
:1013C0007705609078057090790580906E05909013
:1013D0006F05A0907005B090710561C0039709F08A
:1013E0005EC0222309F443C0C0906E05D0906F0503
:1013F000E0907005F090710540907605509077056B
:1014000060907805709079058090720590907305D2
:10141000A0907405B090750542C0C0906605D0904C
:101420006705E0906805F09069054090620550906E
:101430006305609064057090650510C0C0906205FA
:10144000D0906305E0906405F090650540906605D6
:1014500050906705609068057090690580905E0502
:1014600090905F05A0906005B090610518C0C09095
:101470005E05D0905F05E0906005F09061054090BA
:1014800066055090670560906805709069058090CA
:10149000620590906305A0906405B0906505A30176
:1014A0009201C701B6010E94F32929813A814B813B
:1014B0005C810E94A72B1816F4F0A5019401C701C6
:1014C000B6010E94F32929813A814B815C810E94F7
:1014D000A72B181614F080E00FC020910B0130915B
:1014E0000C0140910D0150910E01C701B6010E94FF
:1014F000A72B181684F781E00F900F900F900F9094
:10150000DF91CF91FF90EF90DF90CF90BF90AF90A1
:101510009F908F907F906F905F904F900895AF92C3
:10152000BF92CF92DF92EF92FF920F931F93CF93D0
:10153000DF938091DD059091DE05A091DF05B091EC
:10154000E00540913601509137016091380170916A
:1015500039016C017D01C41AD50AE60AF70A4091E7
:10156000AF055091B0056091B1057091B2054C1571
:101570005D056E057F0508F0F5C08093AF0590937B
:10158000B005A093B105B093B20584EC99E0A0E05A
:10159000B0E08093360190933701A0933801B09367
:1015A000390110919E05D0919D05C0919C0521E0C7
:1015B0004DEC5CEC6CE47DE381E090E00E94A209DC
:1015C000AA24A394811101C0A12C21E04DEC5CEC74
:1015D0006CE47DE382E090E00E94A209BB24B39416
:1015E000811101C0B12C21E04DEC5CEC6CE47DE399
:1015F00083E090E00E94A20901E0811101C000E0B7
:10160000AA2031F1C0907605D0907705E09078055A
:10161000F090790520917205309173054091740521
:1016200050917505C701B6010E94582A87FF0EC068
:1016300020916E0530916F054091700550917105B4
:10164000C701B6010E94582A87FD02C061E001C0AF
:1016500060E081E090E00E941209BB2031F1C0906F
:101660007205D0907305E0907405F0907505209197
:101670007605309177054091780550917905C7013D
:10168000B6010E94582A87FF0EC020916E05309146
:101690006F054091700550917105C701B6010E9418
:1016A000582A87FD02C061E001C060E082E090E05E
:1016B0000E941209002339F1C0906E05D0906F0589
:1016C000E0907005F09071052091760530917705D6
:1016D0004091780550917905C701B6010E94582ABA
:1016E00087FF0EC0209172053091730540917405FB
:1016F00050917505C701B6010E94582A87FD03C0A5
:101700000E948B0105C060E083E090E00E94120916
:10171000A11004C0B11002C0002361F080E29EE479
:10172000A0E0B0E08093360190933701A093380198
:10173000B093390180919E05811308C080919D0569
:101740008D1304C080919C058C1761F0DF91CF91BF
:101750001F910F91FF90EF90DF90CF90BF90AF90CF
:101760000C947504DF91CF911F910F91FF90EF9032
:10177000DF90CF90BF90AF90089520918205309177
:10178000830540918405509185056091860570918F
:10179000870580918805909189050E94F429209100
:1017A0007E0530917F0540918005509181050E9412
:1017B000F4299B01AC0160917A0570917B058091C1
:1017C0007C0590917D050E94A72B18161CF5809131
:1017D0000F0190911001019729F180914505909199
:1017E00046058230910584F0109246051092450519
:1017F00081E090E09093100180930F0162EE71E020
:101800008BEE95E00C9411280196909346058093F9
:101810004505089510924605109245051092100155
:1018200010920F0108951F93CF93DF93192FEB01AF
:10183000482F81EE95E00E948723BE016F5F7F4FA6
:10184000412F81EE95E0DF91CF911F910C9487237A
:101850001F93CF93DF93EC01BC0181EE95E00E94D2
:101860008423182FBE016F5F7F4F81EE95E00E94A9
:101870008423612FDF91CF911F910C947A2761E02F
:101880008DE00E94482560E07DE780E090E00E94C6
:10189000042460E08DE00E94482560E07DE780E060
:1018A00090E00E94042461E08DE00E94482560E001
:1018B0007DE780E090E00E94042460E08DE00E94DB
:1018C000482560E07DE780E090E00E94042461E02C
:1018D0008DE00E94482560E07DE780E090E00E9476
:1018E000042460E08DE00E94482560E07DE780E010
:1018F00090E00C94042461E083E00E9448258091EC
:101900005505882331F06EEE71E08BEE95E00C9476
:101910001128089560E082E00E94482580910A0124
:1019200081110AC080915505882331F064E072E08E
:101930008BEE95E00E94112881E080930A010895C2
:101940008F929F92AF92BF92CF92DF92EF92FF92CF
:10195000CF93DF938091DD059091DE05A091DF05A7
:10196000B091E0058093D5059093D605A093D70557
:10197000B093D8058EE00E946A242091960530919C
:101980009705280F391F30939705209396058FE010
:101990000E946A242091940530919505280F391FE3
:1019A000309395052093940580E10E946A2420914C
:1019B000920530919305280F391F3093930520939A
:1019C000920581E10E946A24EC01209190053091FA
:1019D0009105280F391F309391052093900582E1DE
:1019E0000E946A247C0120918E0530918F05280F7A
:1019F000391F30938F0520938E0520919A053091E1
:101A00009B052F5F3F4F30939B0520939A05BE01A6
:101A1000882777FD8095982F0E94F72A20E030ECE8
:101A20004FE754E40E945C2A2FE632E143E850E499
:101A30000E94AB2B4B015C01B701882777FD809595
:101A4000982F0E94F72A20E030EC4FE754E40E94E0
:101A50005C2A2FE632E143E850E40E94AB2B27E5F5
:101A60003FE348E65EE30E945C2A6B017C012FEFB6
:101A700035EE42E95EE3C501B4010E945C2A9B0198
:101A8000AC01C701B6010E94A72B181684F48091FF
:101A90000A0181110CC0DF91CF91FF90EF90DF9090
:101AA000CF90BF90AF909F908F900C948A0CDF9155
:101AB000CF91FF90EF90DF90CF90BF90AF909F902D
:101AC0008F90089561E082E00E94482510920A01FB
:101AD00080915505882331F06EE172E08BEE95E040
:101AE0000C941128089586E696E6A6E7B0E4809364
:101AF000320190933301A0933401B093350183E315
:101B000093E3A3E7B0E48093AB059093AC05A09377
:101B1000AD05B093AE0580E090E0A0E6B0E4809320
:101B2000220190932301A0932401B09325018DEC11
:101B30009CECACE5B0E480930B0190930C01A09376
:101B40000D01B0930E0180E090E0A0E0BFE3809330
:101B50002E0190932F01A0933001B093310108958D
:101B60008DEC9CECA4E8B0E48093320190933301B7
:101B7000A0933401B093350183E393E3A3E8B0E489
:101B80008093AB059093AC05A093AD05B093AE05E3
:101B900083E393E3A3E7B0E48093220190932301CE
:101BA000A0932401B09325018DEC9CECACE4B0E44F
:101BB00080930B0190930C01A0930D01B0930E0143
:101BC00080E090E0A0E8BFE380932E0190932F0186
:101BD000A0933001B09331010895FF920F931F93AA
:101BE000CF93DF9366E372E08BEE95E00E94E227ED
:101BF00080911F0190912001449721F0C4E1D0E031
:101C0000F12C19C064E472E038C0CE010E94280CA7
:101C10008C01FF2031F067E472E08BEE95E00E94CA
:101C2000E2274AE050E0B8018BEE95E00E94C6281A
:101C30002296FF24F39420911F013091200121501E
:101C40003109C217D3070CF38091530590915405C5
:101C50000817190781F067E472E08BEE95E00E94A7
:101C6000E22760915305709154054AE050E08BEEF5
:101C700095E00E94C62865E472E08BEE95E0DF9166
:101C8000CF911F910F91FF900C94112881309105F5
:101C900019F11CF4892B41F0089582309105A9F1C6
:101CA000039709F484C0089580911805909119054F
:101CB000892B09F4EFC08091530590915405892B2D
:101CC00009F0E8C0109219051092180510921B0532
:101CD00010921A0560E0DBC02091180530911905BB
:101CE0002130310509F4D6C02091530530915405B7
:101CF000232B09F0CFC0909319058093180590937A
:101D00001B0580931A0561E0C2C080911C0590916B
:101D10001D05A0911E05B0911F050097A105B105F5
:101D200039F020911805309119052230310571F0F4
:101D300082E090E0909319058093180581E090E08F
:101D400090931B0580931A0561E021C04091DD0549
:101D50005091DE056091DF057091E0054817590745
:101D60006A077B0708F496C080911A0590911B05BD
:101D7000019729F410921B0510921A0506C081E004
:101D800090E090931B0580931A0560911A058DE0F1
:101D90000E9448258091DD059091DE05A091DF0528
:101DA000B091E005845D9E4FAF4FBF4F36C080912C
:101DB000530590915405892B09F06CC040911C0586
:101DC00050911D0560911E0570911F05411551052B
:101DD0006105710531F080911805909119050397FF
:101DE00029F183E090E0909319058093180581E034
:101DF00090E090931B0580931A0561E08DE00E94AE
:101E000048258091DD059091DE05A091DF05B09118
:101E1000E0058A5B9F4FAF4FBF4F80931C059093A7
:101E20001D05A0931E05B0931F0508958091DD0543
:101E30009091DE05A091DF05B091E005841795072C
:101E4000A607B70738F120911A0530911B052130FC
:101E5000310549F410921B0510921A0584529A4FCD
:101E6000AF4FBF4F0AC021E030E030931B052093F5
:101E70001A058A5B9F4FAF4FBF4F80931C0590930D
:101E80001D05A0931E05B0931F0560911A058DE0F6
:101E90000C94482508950E9446091092B70580E0E9
:101EA00090E00C94460E80913E0581111FC00E9467
:101EB0004B0F69E472E08BEE95E00E94112880914F
:101EC000DD059091DE05A091DF05B091E00580531E
:101ED000984FAF4FBF4F8093410590934205A09319
:101EE0004305B093440581E080933E050895CF9368
:101EF000DF93C4E1D0E080911F01909120018C1705
:101F00009D073CF0CE010E94280C889704F522968C
:101F1000F2CFC4E1D0E080911F01909120010196A1
:101F20008C179D0744F040E0BE0181EE95E00E94D1
:101F300087232196F0CF84E190E090932001809355
:101F40001F0180E090E00E94AB0F81E001C080E0C3
:101F5000DF91CF9108950F931F93CF93DF93EC01FF
:101F600004E110E0C730D10511F4C0E0D0E0809169
:101F7000530590915405C817D907D9F12097C9F195
:101F8000C330D10561F480911F019091200184310B
:101F9000910529F002970E94280C039721F1609186
:101FA0001F0170912001CE010E94130C60911F014E
:101FB000709120016E5F7F4F80E090E00E94130CD3
:101FC00080911F01909120010296909320018093AF
:101FD0001F0180915505882331F064E572E08BEE96
:101FE00095E00E941128D0935405C09353050E9498
:101FF000ED0DD0935405C093530582E090E00E940C
:10200000460E8091530590915405009719F0873042
:10201000910529F480E090E00E94460E23C08431AF
:10202000910504F19C01245131092431310528F432
:102030000E944B0F0E94730D15C09C01285231095C
:102040002431310528F4109221010E944B0F0AC05F
:102050009C012C5331092431310550F380559109ED
:10206000449788F380911F0190912001843A914018
:10207000E4F00E94770F811118C0109320010093A3
:102080001F0164E170E080915305909154050E9416
:10209000130C80911F0190912001029690932001D2
:1020A00080931F01CEE3D0E05DCFDF91CF911F91F0
:1020B0000F9108958F929F92AF92BF92CF92DF922D
:1020C000EF92FF9280E00E94672460E08EE00E9421
:1020D0000F2560E08FE00E940F2560E080E10E9404
:1020E0000F2560E081E10E940F2560E082E10E94FF
:1020F0000F2561E088E00E940F2561E087E00E94E3
:102100000F2561E084E00E940F2560E088E00E94D6
:10211000482561E087E00E94482561E084E00E9454
:10212000482585B5887F816085BD61E08DE00E948E
:102130000F25609118058DE00E94482561E085E03B
:102140000E940F256091C4057091C50585E00E942D
:10215000872461E083E00E940F2561E083E00E9414
:10216000482561E082E00E940F2560E082E00E9445
:10217000482526E040E052EC61E070E08BEE95E00F
:102180000E9418276CE672E08BEE95E00E94112801
:1021900082E090E00E94280C181619067CF4BC011D
:1021A000882777FD8095982F0E94F72A60931B015E
:1021B00070931C0180931D0190931E0180E090E0BC
:1021C0000E94280CBC01882777FD8095982F0E94DB
:1021D000F72A6B017C0180901B0190901C01A0905C
:1021E0001D01B0901E01A50194010E94A72B181695
:1021F0004CF480924F0590925005A0925105B092F8
:10220000520508C0C0924F05D0925005E09251058A
:10221000F092520584E090E00E94280C0097B9F0FB
:10222000BC01685E7340882777FD8095982F0E94D7
:10223000F72A20E030E04AE754E40E945C2A6093E9
:10224000240570932505809326059093270586E045
:1022500090E00E94280CBC01882777FD8095982F7C
:102260000E94F72A20E030E04AE754E40E945C2A0A
:102270006B017C0124E333E347E451E40E94A72B84
:1022800018167CF5C0921101D0921201E092130150
:10229000F09214012AE939E949E15FE3C701B60187
:1022A0000E94F329609334057093350580933605B9
:1022B0009093370516C00E94280C0097D1F0909398
:1022C0005405809353058730910511F00E94AB0FA0
:1022D00080911F019091200102969093200180939C
:1022E0001F0180911F0190912001893B21E09207FD
:1022F00014F3FF90EF90DF90CF90BF90AF909F903E
:102300008F900895CF92DF92EF92FF9220918205F5
:102310003091830540918405509185056091860533
:102320007091870580918805909189050E94F42914
:1023300020917E0530917F05409180055091810567
:102340000E94F4296B017C0120E030E040E450E47D
:1023500060912201709123018091240190912501C7
:102360000E94AB2B9B01AC01C701B6010E94582A09
:1023700087FF18C02DEC3CEC44E850E4609132013A
:102380007091330180913401909135010E94582A57
:10239000811108C08DE290E0FF90EF90DF90CF9028
:1023A0000C94AB0F0E944B0F2DEC3CEC44E850E436
:1023B0006091320170913301809134019091350127
:1023C0000E94582A81111AC080911B0190911C0112
:1023D000A0911D01B0911E0180934F05909350056F
:1023E000A0935105B093520564E772E08BEE95E03F
:1023F000FF90EF90DF90CF900C941128FF90EF901A
:10240000DF90CF900895CF92DF92EF92FF92C0902D
:102410007A05D0907B05E0907C05F0907D052091B9
:102420001101309112014091130150911401C70123
:10243000B6010E94A72B87FD8BC010924A0510920F
:1024400049058091150190911601019709F4ECC09E
:102450008091470590914805823091050CF472C037
:10246000109248051092470581E090E09093160184
:10247000809315016EE772E08BEE95E00E941128C3
:1024800080912101882309F4CFC0C090AB05D09082
:10249000AC05E090AD05F090AE05A7019601609106
:1024A00086057091870580918805909189050E9425
:1024B000A72B87FD22C0A70196016091820570912C
:1024C000830580918405909185050E94A72B87FD47
:1024D00014C0A701960160917E0570917F058091DF
:1024E0008005909181050E94A72B87FD06C0FF9073
:1024F000EF90DF90CF900C94821180915505882346
:1025000031F067E872E08BEE95E00E94112860E1FF
:1025100077E280E090E00E9457098091DD0590917C
:10252000DE05A091DF05B091E00588579C4EAF4FC6
:10253000BF4F8093200590932105A0932205B0936F
:10254000230572C0019690934805809347056CC09F
:10255000109248051092470520918205309183051D
:10256000409184055091850560918605709187059D
:1025700080918805909189050E94F42920917E051B
:1025800030917F0540918005509181050E94F4298A
:102590009B01AC01C701B6010E94582A18160CF421
:1025A0003FC08091150190911601892BE9F180912E
:1025B000490590914A058230910564F110924A05CF
:1025C00010924905109216011092150166E972E009
:1025D0008BEE95E00E9411280E94620D109220055A
:1025E000109221051092220510922305809121015D
:1025F0008823D1F080915505882331F061EA72E09B
:102600008BEE95E00E941128FF90EF90DF90CF9025
:102610000C944B0F019690934A058093490504C092
:1026200010924A0510924905FF90EF90DF90CF90ED
:102630000895CF92DF92EF92FF92C090DD05D09087
:10264000DE05E090DF05F090E005C092B305D09282
:10265000B405E092B505F092B6058091A70590917A
:10266000A805A091A905B091AA05B701A601481B2C
:10267000590B6A0B7B0B80912A0190912B01A09141
:102680002C01B0912D0184179507A607B70778F4A0
:1026900080915505882331F061EB72E08BEE95E077
:1026A0000E9411280E944B0F8EE290E03EC0809164
:1026B000530590915405039731F4FF90EF90DF900C
:1026C000CF900C944B0F24EA30E745E850E460913A
:1026D00076057091770580917805909179050E9433
:1026E000A72B181604F124EA30E745E850E460917E
:1026F00072057091730580917405909175050E9423
:10270000A72B181684F024EA30E745E850E46091DE
:102710006E0570916F0580917005909171050E9412
:10272000A72B181644F48BE290E0FF90EF90DF9017
:10273000CF900C94AB0F2DEC3CEC4CE45EE360913D
:1027400056057091570580915805909159050E9442
:10275000582A87FF23C08091C8058823F9F080910B
:10276000A3059091A405A091A505B091A605C81A4E
:10277000D90AEA0AFB0A8091260190912701A091CB
:102780002801B09129018C159D05AE05BF0570F497
:10279000FF90EF90DF90CF900C948211C092A30530
:1027A000D092A405E092A505F092A60581E090E004
:1027B0000E94460EC0902E01D0902F01E090300173
:1027C000F09031012DEC3CEC4CE450E46091760546
:1027D0007091770580917805909179050E94582A2B
:1027E00087FD20C02DEC3CEC4CE450E46091720578
:1027F0007091730580917405909175050E94582A17
:1028000087FD10C02DEC3CEC4CE450E460916E056B
:1028100070916F0580917005909171050E94582A02
:1028200087FF31C080915505882331F063EC72E059
:102830008BEE95E00E9411288091DD059091DE05D8
:10284000A091DF05B091E0054091A7055091A80542
:102850006091A9057091AA05841B950BA60BB70B77
:1028600081309D4DAD46B10518F08DE290E05DCF11
:1028700085E090E00E94AB0F8AE9C82E89E9D82E46
:10288000ED2C8EE3F82E29E23CE54FE05EE3C70134
:10289000B6010E94F3299B01AC016091560570912D
:1028A000570580915805909159050E94A72B87FDE7
:1028B0003CC02AE037ED43EA5CE360919F057091EC
:1028C000A0058091A1059091A2050E94F429209174
:1028D00032013091330140913401509135010E9411
:1028E000582A181614F1A7019601609144017091BD
:1028F000450180914601909147010E94582A81111B
:1029000004C08091C705811102C00E947504C09265
:102910004401D0924501E0924601F092470181E0E6
:102920008093C7051092C80531C02AE037ED43E215
:102930005CE3609132017091330180913401909198
:1029400035010E94F3296B017C019B01AC01609170
:1029500048017091490180914A0190914B010E9478
:10296000582A811104C08091C805811102C00E94BB
:102970007504C0924801D0924901E0924A01F09258
:102980004B0181E08093C8051092C7058091C60570
:10299000811106C0FF90EF90DF90CF900C948F0ACA
:1029A000FF90EF90DF90CF9008958F929F92AF921B
:1029B000BF92CF92DF92EF92FF9210922005109279
:1029C0002105109222051092230580910A01882387
:1029D000D9F08091C4059091C50518161906A4F088
:1029E00020913405309135054091360550913705D9
:1029F00060917A0570917B0580917C0590917D05B1
:102A00000E94582A87FF03C081E090E04CC080906C
:102A1000240590902505A0902605B0902705A501D6
:102A2000940160918A0570918B0580918C0590913D
:102A30008D050E94F3299B01AC0168E17AEF88E2E1
:102A40009BEB0E94F3296B017C016093240570933A
:102A50002505809326059093270520E030E0A90105
:102A60000E94A72B18165CF42DEC3CEC4CEC5EE3BA
:102A7000C701B6010E94A72B18165CF01EC02DECF2
:102A80003CEC4CEC5EEBC701B6010E94582A87FF74
:102A900014C08092240590922505A0922605B0923C
:102AA000270581E590E0FF90EF90DF90CF90BF90F9
:102AB000AF909F908F900C94AB0F80915505882319
:102AC00041F165ED72E08BEE95E00E9411282091B6
:102AD0002405309125054091260550912705C50113
:102AE000B4010E94582A8823A1F064EE72E08BEEB4
:102AF00095E00E94E22740912405509125056091C0
:102B000026057091270522E030E08BEE95E00E94CB
:102B1000E02920E030E04AE754E460912405709118
:102B2000250580912605909127050E94AB2B20E07A
:102B300030E04AE754E40E94F4290E94C42ADC01F0
:102B4000CB0164E070E0FF90EF90DF90CF90BF90FA
:102B5000AF909F908F900C94130C60E083E00E94E4
:102B6000482580915505882331F066EF72E08BEEA1
:102B700095E00E941128809115019091160101970E
:102B800051F060E072EE84E090E00E9404248DE356
:102B900090E00C94AB0F0895CF92DF92EF92FF92EA
:102BA0008091150190911601892B09F0FEC0C0900B
:102BB0000B01D0900C01E0900D01F0900E01A701E7
:102BC00096016091860570918705809188059091A6
:102BD00089050E94582A87FD1CC0A70196016091B3
:102BE00082057091830580918405909185050E94EE
:102BF000582A87FD0EC0A701960160917E0570914D
:102C00007F0580918005909181050E94582A87FF59
:102C100036C080913F0590914005803591054CF17B
:102C20001092400510923F050E94530F2DEC3CEC92
:102C30004CE450E460910B0170910C0180910D0106
:102C400090910E010E94582A81111DC086E090E0EB
:102C50000E94AB0F80915505882309F4A6C06DE052
:102C600073E08BEE95E0FF90EF90DF90CF900C94A7
:102C7000112801969093400580933F0504C010925F
:102C8000400510923F0520E030E040E650E46091BE
:102C900086057091870580918805909189050E942D
:102CA000582A87FD20C020E030E040E650E46091E3
:102CB00082057091830580918405909185050E941D
:102CC000582A87FD10C020E030E040E650E46091D3
:102CD0007E0570917F0580918005909181050E940D
:102CE000582A87FF5EC0809138059091390580355C
:102CF00091050CF450C0109239051092380580915E
:102D00001805909119050397F1F120914F05309125
:102D10005005409151055091520560911B017091F1
:102D20001C0180911D0190911E010E94F32923E353
:102D300033E343E75FE30E945C2A60931B017093D7
:102D40001C0180931D0190931E010E94C42ADC0186
:102D5000CB0162E070E00E94130C2DEC3CEC4CE4E3
:102D60005DE360911B0170911C0180911D019091A8
:102D70001E010E94AB2B60934F057093500580930A
:102D800051059093520583E090E0FF90EF90DF9023
:102D9000CF900C94460E0196909339058093380598
:102DA00004C01092390510923805FF90EF90DF9023
:102DB000CF9008952091820530918305409184053C
:102DC00050918505609186057091870580918805F1
:102DD000909189050E94F4292DEC3CEC4CE45EE3D3
:102DE0000E94582A87FF06C083E090E00E94AB0F44
:102DF0000C944B0F8091530590915405039721F447
:102E000080E090E00C94AB0F0895809115019091B3
:102E10001601019729F0109233051092320508959A
:102E20002091340530913505409136055091370594
:102E300060917A0570917B0580917C0590917D056C
:102E40000E94582A87FFE7CF809132059091330581
:102E50008A30910584F0109233051092320562E2B7
:102E600073E08BEE95E00E9411280E944B0F84E0E6
:102E700090E00C94AB0F019690933305809332054C
:102E8000089526E636E646EE5EE360918A05709187
:102E90008B0580918C0590918D050E94A72B1816AB
:102EA000D4F48091C4059091C505892BA1F480913B
:102EB000300590913105853091053CF082E590E038
:102EC0000E94AB0F0E948A0C06C0019690933105B8
:102ED00080933005089510923105109230050895C1
:102EE00020E030E040E05FE360918A0570918B055F
:102EF00080918C0590918D050E94582A87FF19C0FA
:102F00008091C4059091C505843B910591F4809111
:102F10002A0590912B05893291052CF08AE290E0E8
:102F20000E94AB0F06C0019690932B0580932A0553
:102F3000089510922B0510922A05089520912E01D4
:102F400030912F01409130015091310160918A05FB
:102F500070918B0580918C0590918D050E94F329CD
:102F600029E23CE54FE05EE30E94A72B181694F49B
:102F70008091280590912905853191052CF083E5F4
:102F800090E00E94AB0F06C00196909329058093B4
:102F9000280508951092290510922805089520E02B
:102FA00030E040E750EC60918A0570918B0580918C
:102FB0008C0590918D050E94582A87FF17C080913B
:102FC0003C0590913D05833091055CF06BE273E028
:102FD0008BEE95E00E94112810923D0510923C0561
:102FE00005C0019690933D0580933C0520E030E0BC
:102FF00048E850EC60918A0570918B0580918C05B2
:1030000090918D050E94582A87FF17C080913A053C
:1030100090913B05833091055CF082E090E00E9446
:10302000AB0F0E94AD1510923B0510923A05089522
:10303000019690933B0580933A050895CF93DF93D3
:1030400000D0CDB7DEB720918806309189062115D2
:10305000310511F42CE836E0CE010196821B930B6A
:103060000F900F90DF91CF9108958091DD059091A1
:10307000DE05A091DF05B091E0058093D90590931E
:10308000DA05A093DB05B093DC058091B8058111CA
:1030900071C06EE572E08BEE95E00E94BD27409115
:1030A0008A0550918B0560918C0570918D0522E009
:1030B00030E08BEE95E00E94E02964E572E08BEE53
:1030C00095E00E94BD27409186055091870560914B
:1030D00088057091890522E030E08BEE95E00E9432
:1030E000E0296AE472E08BEE95E00E94BD274091F2
:1030F000820550918305609184057091850522E0D9
:1031000030E08BEE95E00E94E02960E472E08BEE07
:1031100095E00E94BD2740917E0550917F0560910A
:1031200080057091810522E030E08BEE95E00E94F1
:10313000E02962E372E08BEE95E00E94BD272091CA
:1031400082053091830540918405509185056091F9
:1031500086057091870580918805909189050E9468
:10316000F42920917E0530917F0540918005509192
:103170008105D6C06AE172E08BEE95E00E94BD2722
:103180004091560550915705609158057091590529
:1031900022E030E08BEE95E00E94E02967E072E0EB
:1031A0008BEE95E00E94BD27409166055091670522
:1031B000609168057091690522E030E08BEE95E042
:1031C0000E94E02964EF71E08BEE95E00E94BD273C
:1031D00040916205509163056091640570916505A9
:1031E00022E030E08BEE95E00E94E02961EE71E094
:1031F0008BEE95E00E94BD2740915E0550915F05E2
:10320000609160057091610522E030E08BEE95E001
:103210000E94E0296AEC71E08BEE95E00E94BD27E8
:1032200020916205309163054091640550916505D8
:1032300060916605709167058091680590916905B8
:103240000E94F42920915E0530915F054091600550
:10325000509161050E94F429AB01BC0122E030E0ED
:103260008BEE95E00E94E0296BEB71E08BEE95E030
:103270000E94BD27409176055091770560917805B1
:103280007091790522E030E08BEE95E00E94E02914
:103290006CEA71E08BEE95E00E94BD2740917205CB
:1032A00050917305609174057091750522E030E0CE
:1032B0008BEE95E00E94E0296DE971E08BEE95E0E0
:1032C0000E94BD2740916E0550916F056091700579
:1032D0007091710522E030E08BEE95E00E94E029CC
:1032E0006AE871E08BEE95E00E94BD27209172059F
:1032F0003091730540917405509175056091760584
:103300007091770580917805909179050E94F42954
:1033100020916E0530916F054091700550917105B7
:103320000E94F429AB01BC0122E030E08BEE95E075
:103330000E94E02961E871E08BEE95E00E94BD27D4
:103340006091C4057091C5054AE050E08BEE95E0B0
:103350000E94CE2862E771E08BEE95E00E94BD27C7
:10336000409148015091490160914A0170914B018F
:1033700022E030E08BEE95E00E94E02964E671E007
:103380008BEE95E00E94BD2740914401509145018C
:10339000609146017091470122E030E08BEE95E0AC
:1033A0000E94E02980919E05882341F065E571E047
:1033B0008BEE95E00E94BD2781E001C080E09091F6
:1033C0009D05992339F066E471E08BEE95E00E944B
:1033D000BD2781E090919C05992339F067E371E066
:1033E0008BEE95E00E94BD2781E09091C80599235E
:1033F00039F06AE271E08BEE95E00E94BD2781E032
:103400009091C705992339F06EE171E08BEE95E05C
:103410000E94BD2781E09091C605992339F063E1B0
:1034200071E08BEE95E00E94BD2702C0882331F049
:1034300062EC72E08BEE95E00E94112861E171E090
:103440008BEE95E00E94BD274091DD055091DE0591
:103450006091DF057091E0052AE030E08BEE95E0A9
:103460000E94E6286FE071E08BEE95E00E94BD2798
:103470008091B805882309F445C0409156055091C4
:103480005705609158057091590522E030E08BEEA8
:1034900095E00E94DE296DE071E08BEE95E00E94E0
:1034A000BD27409166055091670560916805709150
:1034B000690522E030E08BEE95E00E94DE296BE0AA
:1034C00071E08BEE95E00E94BD274091620550911E
:1034D0006305609164057091650522E030E08BEE34
:1034E00095E00E94DE2969E071E08BEE95E00E9494
:1034F000BD2740915E0550915F0560916005709118
:10350000610544C040918A0550918B0560918C05FE
:1035100070918D0522E030E08BEE95E00E94DE296F
:1035200067E071E08BEE95E00E94BD274091860533
:1035300050918705609188057091890522E030E0FF
:103540008BEE95E00E94DE2965E071E08BEE95E060
:103550000E94BD27409182055091830560918405AA
:103560007091850522E030E08BEE95E00E94DE2927
:1035700063E071E08BEE95E00E94BD2740917E05EF
:1035800050917F05609180057091810522E030E0C7
:103590008BEE95E00E94DE2961E071E08BEE95E014
:1035A0000E94BD2740917A0550917B0560917C0572
:1035B00070917D0522E030E08BEE95E00E94DE29DF
:1035C0006FEF70E08BEE95E00E94BD276091C4051F
:1035D0007091C5054AE050E08BEE95E00E94C62848
:1035E0006DEF70E08BEE95E00E94FF276FEE70E0CC
:1035F0008BEE95E00E94BD2760919805709199052A
:103600004AE050E08BEE95E00E94CE286CED70E031
:103610008BEE95E00E94BD27409124055091250531
:10362000609126057091270522E030E08BEE95E051
:103630000E94E02980910A01882319F06CEC70E067
:1036400002C06DEB70E08BEE95E00E94FF27809149
:10365000B805882319F16CEA70E08BEE95E00E94C2
:10366000BD2740916A0550916B0560916C05709182
:103670006D0522E030E08BEE95E00E94E02967E9DD
:1036800070E08BEE95E00E94BD2740915A05509165
:103690005B0560915C0570915D050EC06BE870E0A4
:1036A0008BEE95E00E94BD2740917A0550917B05F5
:1036B00060917C0570917D0522E030E08BEE95E015
:1036C0000E94E0298091530590915405892B81F047
:1036D00063E870E08BEE95E00E94BD276091530592
:1036E000709154054AE050E08BEE95E00E94CE28A0
:1036F00068E770E08BEE95E00E94BD270E941E18DF
:103700004AE050E0BC018BEE95E00E94CE2862ECCE
:1037100072E08BEE95E00C94112868E670E08BEE79
:1037200095E00C94FF27CF92DF92EF92FF92CF9318
:10373000DF93C0910805D0910905C133D10501F58A
:1037400062EC72E08BEE95E00E94112880919E055C
:10375000882341F06AE373E08BEE95E00E94112824
:1037600060E007C065E473E08BEE95E00E941128ED
:1037700061E081E090E00E94120962EC72E086C490
:10378000C233D105F1F462EC72E08BEE95E00E9459
:10379000112880919D05882341F06FE473E08BEE42
:1037A00095E00E94112860E007C06AE573E08BEEA7
:1037B00095E00E94112861E082E090E00E941209E9
:1037C000AFC1C333D105E9F462EC72E08BEE95E052
:1037D0000E94112880919C05882351F064E673E0D3
:1037E0008BEE95E00E94112860E083E090E0E6CF48
:1037F0006FE673E08BEE95E00E9411280E948B012A
:103800008FC1C033D10529F560E088E00E944825CA
:1038100061E087E00E94482561E084E00E9448253D
:1038200062EC72E08BEE95E00E94112869E773E08C
:103830008BEE95E00E94112862EC72E08BEE95E031
:103840000E94112810929E0510929D0510929C05D1
:10385000E0C1C136D105F1F460E070E085E00E947E
:10386000872462EC72E08BEE95E00E94112868E8F4
:1038700073E08BEE95E00E94112862EC72E08BEE13
:1038800095E00E9411281092C5051092C40560E0D1
:1038900070E096C1C236D10501F564E670E085E0BE
:1038A0000E94872462EC72E08BEE95E00E94112862
:1038B00064E973E08BEE95E00E94112862EC72E0FF
:1038C0008BEE95E00E94112884E690E09093C50568
:1038D0008093C40564E670E073C1C336D10501F579
:1038E00068EC70E085E00E94872462EC72E08BEE69
:1038F00095E00E94112862EA73E08BEE95E00E9449
:10390000112862EC72E08BEE95E00E94112888ECA1
:1039100090E09093C5058093C40568EC70E050C1B9
:10392000C436D10501F56FEF70E085E00E94872471
:1039300062EC72E08BEE95E00E94112860EB73E080
:103940008BEE95E00E94112862EC72E08BEE95E020
:103950000E9411288FEF90E09093C5058093C405D5
:103960006FEF70E02DC1C536D105F9F462EC72E05D
:103970008BEE95E00E9411288091C805882349F0BC
:103980001092C8056EEB73E08BEE95E00E94E22783
:10399000C7C081E08093C8056BEC73E08BEE95E0C7
:1039A0000E94E2270E947504BBC0C636D10569F5A6
:1039B00062EC72E08BEE95E00E9411288091C705C1
:1039C000882349F01092C70567ED73E08BEE95E010
:1039D0000E94E2270BC081E08093C70563EE73E08D
:1039E0008BEE95E00E94E2270E94750462EC72E083
:1039F0008BEE95E00E9411281092D1051092D2050D
:103A00001092D3051092D40504C1C937D105F9F439
:103A10002DEC3CEC4CE45DE3609144017091450178
:103A200080914601909147010E94F42960934401DE
:103A300070934501809346019093470162EC72E0D8
:103A40008BEE95E00E9411286EEE73E065C0C836DB
:103A5000D105F9F42DEC3CEC4CE45DE360914401BC
:103A60007091450180914601909147010E94F32990
:103A70006093440170934501809346019093470100
:103A800062EC72E08BEE95E00E94112860E074E039
:103A900043C0C537D105F9F42AE037ED43EA5CE3CA
:103AA000609148017091490180914A0190914B01C8
:103AB0000E94F429609348017093490180934A0160
:103AC00090934B0162EC72E08BEE95E00E9411281E
:103AD00062E174E021C0CA36D10549F52AE037ED2C
:103AE00043EA5CE3609148017091490180914A0189
:103AF00090914B010E94F329609348017093490112
:103B000080934A0190934B0162EC72E08BEE95E05A
:103B10000E94112865E274E08BEE95E00E94112866
:103B200062EC72E08BEE95E00E94112872C0C936FB
:103B3000D10511F562EC72E08BEE95E00E94112840
:103B40006AE374E08BEE95E00E94112862EC72E06B
:103B50008BEE95E00E9411288091C4059091C505D7
:103B60000A968F3F910519F014F08FEF90E0909333
:103B7000C5058093C40520C0CB36D10529F562EC7C
:103B800072E08BEE95E00E94112865E474E08BEE04
:103B900095E00E94112862EC72E08BEE95E00E94A5
:103BA00011288091C4059091C5050A9797FFDFCF32
:103BB0001092C5051092C4056091C4057091C505A9
:103BC00085E00E94872425C0CF36D10511F562EC2F
:103BD00072E08BEE95E00E94112860E574E08BEEB8
:103BE00095E00E94112862EC72E08BEE95E00E9455
:103BF00011288091C4059091C50501968F3F9105CC
:103C000019F014F08FEF90E09093C5058093C405F0
:103C100020C0CC36D10551F562EC72E08BEE95E018
:103C20000E9411286AE574E08BEE95E00E9411284D
:103C300062EC72E08BEE95E00E9411288091C40541
:103C40009091C505019797FFDFCF1092C50510929F
:103C5000C4056091C4057091C50585E0DF91CF91E1
:103C6000FF90EF90DF90CF900C948724C736D1055A
:103C7000F9F462EC72E08BEE95E00E9411288091DD
:103C8000B705882349F061EA72E08BEE95E00E9467
:103C900011280E944B0F71CD67E872E08BEE95E022
:103CA0000E94112860E070E0CB010E94570965CDA9
:103CB000CA37D10541F4DF91CF91FF90EF90DF90AB
:103CC000CF900C94D514C637D10579F48091210199
:103CD000882329F01092210164E674E0D7C181E0C5
:103CE0008093210161E774E0D1C1C837D10519F48F
:103CF0006DE774E0CBC1C137D10559F4809155050A
:103D0000882319F010925505CBC181E080935505A9
:103D1000C7C1C237D10541F4DF91CF91FF90EF9039
:103D2000DF90CF900C94AD15C437D10541F4DF91ED
:103D3000CF91FF90EF90DF90CF900C947B0CCD361D
:103D4000D10541F4DF91CF91FF90EF90DF90CF90BC
:103D50000C948A0CCE36D10541F4DF91CF91FF90BF
:103D6000EF90DF90CF900C94620DC037D10541F4F5
:103D7000DF91CF91FF90EF90DF90CF900C94530F95
:103D8000C737D105A9F48091DD059091DE05A0919A
:103D9000DF05B091E005805A9541AF4FBF4F80934A
:103DA000410590934205A0934305B093440578C123
:103DB000C337D10529F1C433D105E9F480E090E09F
:103DC0000E94AB0FC4E1D0E080911F0190912001CF
:103DD00001968C179D0744F040E0BE0181EE95E00E
:103DE0000E9487232196F0CF84E190E090932001F8
:103DF00080931F0105C0C234D10551F40E94770F92
:103E0000DF91CF91FF90EF90DF90CF900C94ED0D6C
:103E1000C334D10509F5809153059091540501975C
:103E2000879770F780911F0190912001449741F38B
:103E300080E090E00E94AB0F60911F017091200123
:103E4000625071097093200160931F0140E081EE80
:103E500095E00E948723D4CFC533D105D1F460917A
:103E60000A0580910C050E947A27EC01BC0180E0D4
:103E700090E00E94F52A60931B0170931C018093CF
:103E80001D0190931E0162E070E0CE010E94130CB0
:103E900003C0C633D10579F46FE874E08BEE95E08A
:103EA0000E94E22740911B0150911C0160911D016D
:103EB00070911E01E3C0C634D10589F560910A05F1
:103EC00070910B05882777FD8095982F0E94F72A1F
:103ED00020911B0130911C0140911D0150911E0148
:103EE0000E94AB2B20E030E048EC52E40E945C2AB8
:103EF00060934F0570935005809351059093520540
:103F00006EE974E08BEE95E00E94E22740914F0548
:103F1000509150056091510570915205AFC0C73363
:103F2000D10541F4DF91CF91FF90EF90DF90CF90DA
:103F30000C948D1BC833D10581F4C0E0D0E040E083
:103F4000BE0181EE95E00E9487232196C11582E093
:103F5000D807A9F765EA74E099C0C933D105B9F467
:103F600060910A058091060590910705039719F461
:103F700080910C0501C080E00E947A27EC010E942C
:103F8000AB0F249709F08CC062E273E07FC0C134AC
:103F9000D10519F560914F0570915005809151053B
:103FA000909152050E94C42ADC01CB0160E070E0D0
:103FB0000E94130C8091DD059091DE05A091DF0534
:103FC000B091E00580934B0590934C05A0934D056F
:103FD000B0934E0565EB74E059C0C434D105E9F5E2
:103FE00060910A0580910C050E947A27EC01BC01C2
:103FF000882777FD8095982F0E94F72A20E030E0EF
:104000004AE754E40E945C2A6B017C0124E333E319
:1040100047E451E40E94A72B18160CF041C0C0924F
:104020001101D0921201E0921301F09214012AE9D9
:1040300039E949E15FE3C701B6010E94F3296093C2
:10404000340570933505809336059093370566E007
:1040500070E0CE010E94130C03C0C534D10501F5F8
:1040600069EC74E08BEE95E00E94E227409111012B
:1040700050911201609113017091140122E030E01F
:104080008BEE95E00E94DE2965E472E08BEE95E010
:10409000DF91CF91FF90EF90DF90CF900C9411289B
:1040A000DF91CF91FF90EF90DF90CF9008952DECAE
:1040B0003CEC4CE45DE360913201709133018091FE
:1040C0003401909135010E94F3296093AB05709300
:1040D000AC058093AD059093AE052AE939E949E135
:1040E0005FE3609111017091120180911301909131
:1040F00014010E94F3296093340570933505809371
:1041000036059093370508958BEE95E00E944E2674
:1041100060910605709107059B012F5F3F4F30931B
:10412000070520930605FB01EE0FFF1FE85FFA4F1E
:104130009183808340910805509109058D30910548
:1041400019F08A30910571F44533510559F0443422
:10415000510541F0121613062CF470930705609375
:10416000060509C04533510519F04434510531F4B1
:104170002330310519F40E94931B08C08D3091053E
:1041800011F00A9739F42130310521F41092070516
:10419000109206058091DD059091DE05A091DF0566
:1041A000B091E00580932C0590932D05A0932E05EA
:1041B000B0932F058091530590915405079731F4E2
:1041C00080E090E00E94AB0F0C94B00D08958F92A8
:1041D0009F92AF92BF92CF92DF92EF92FF920F9396
:1041E0001F930E94D5230E94F52A20E030E040E88A
:1041F0005CE30E94AB2B0E94C92A0091DD0510915F
:10420000DE052091DF053091E00560177107820718
:10421000930740F46093BE057093BF058093C0057B
:104220009093C1056093DD057093DE058093DF05F3
:104230009093E00520919E0521111BC020919D05C2
:10424000211117C020919C05211113C02091C40594
:104250003091C5051216130664F02091C80521118E
:1042600008C02091C705211104C02091B705222361
:1042700021F021E02093B80502C01092B80500910A
:104280003E0110913F0120914001309141014B01CD
:104290005C01801A910AA20AB30AC090BA05D090B4
:1042A000BB05E090BC05F090BD05C814D904EA0434
:1042B000FB0450F4601771078207930728F0809180
:1042C000B80581110E94C5018091DD059091DE0540
:1042D000A091DF05B091E0058C019D010A5F1109F5
:1042E000210931094091D1055091D2056091D30542
:1042F0007091D405401751076207730700F58A3F94
:104300009105A105B105D8F080919A0590919B0582
:1043100018161906A4F40E94B3040E9403120E9406
:10432000BD0B0E94CC150E94DA160E9405170E9450
:1043300041170E9470170E949E170E94CF1780910C
:10434000DD059091DE05A091DF05B091E0058C01BF
:104350009D01005D1740210931094091D905509117
:10436000DA056091DB057091DC05401751076207A3
:104370007307B8F4803D9740A105B10590F0809196
:104380003E0190913F01A0914001B0914101883CD4
:104390009105A105B10529F08091550581110E9473
:1043A00035188091DD059091DE05A091DF05B09173
:1043B000E0058C019D010A5F110921093109409135
:1043C000C9055091CA056091CB057091CC05401785
:1043D00051076207730770F48A3F9105A105B10583
:1043E00048F08091C805811103C08091C7058111F3
:1043F0000E947F078091DD059091DE05A091DF0589
:10440000B091E0058C019D01045C1940210931093E
:104410004091B3055091B4056091B5057091B60512
:10442000401751076207730750F4843C9940A10577
:10443000B10528F08091B70581110E941913809170
:10444000DD059091DE05A091DF05B091E0058C01BE
:104450009D0108581341210931094091CD05509122
:10446000CE056091CF057091D005401751076207C6
:104470007307C0F488389341A105B10598F0809185
:104480003E0190913F01A0914001B0914101883CD3
:104490009105A105B10531F080915505811102C04A
:1044A0000E9453028091DD059091DE05A091DF0509
:1044B000B091E0058C019D01005E13492440310953
:1044C00040914B0550914C0560914D0570914E0502
:1044D0004017510762077307F8F4803E23E99207FB
:1044E00024E0A207B105C0F080934B0590934C05E2
:1044F000A0934D05B0934E0560914F057091500506
:1045000080915105909152050E94C42ADC01CB0193
:1045100060E070E00E94130C8091200590912105CD
:10452000A0912205B09123054091DD055091DE0553
:104530006091DF057091E00584179507A607B7071E
:1045400030F4892B8A2B8B2B11F00E94D51480918B
:104550001805909119050E94460E8091DD059091F5
:10456000DE05A091DF05B091E0058C019D010058AA
:104570001F442241310940912C0550912D05609135
:104580002E0570912F05401751076207730798F4A5
:1045900080382FE4920722E1A207B10560F08093F2
:1045A0002C0590932D05A0932E05B0932F0587E041
:1045B00090E00E94AB0F8091DD059091DE05A09107
:1045C000DF05B091E0054091BE055091BF056091B7
:1045D000C0057091C105841B950BA60BB70B813CE0
:1045E000944DA140B10540F08091C605882321F08B
:1045F0008CE290E00E94AB0F4091DD055091DE050A
:104600006091DF057091E00580914C0190914D0122
:10461000A0914E01B0914F016A017B01C81AD90ADD
:10462000EA0AFB0A0091D5051091D6052091D7051D
:104630003091D8050C151D052E053F0538F4481797
:1046400059076A077B0710F00E94A00C8BEE95E0DB
:104650000E943326181619066CF480913E01909141
:104660003F01A0914001B0914101883C9105A10515
:10467000B105E1F58091410590914205A091430576
:10468000B09144050097A105B10599F14091DD0570
:104690005091DE056091DF057091E00548175907DC
:1046A0006A077B0730F160914F057091500580914A
:1046B0005105909152050E94C42ADC01CB0160E0B3
:1046C00070E00E94130C0E943F0C0E94AD1568ED33
:1046D00074E08BEE95E00E94112810924105109233
:1046E0004205109243051092440503C00E948420A5
:1046F000C1CF1F910F91FF90EF90DF90CF90BF90AF
:10470000AF909F908F900895CB010C94622CCB01B9
:10471000642F0C946A2C1F920F920FB60F921124E3
:104720002F933F938F939F93AF93BF938091E30514
:104730009091E405A091E505B091E6053091E20580
:1047400023E0230F2D3720F40196A11DB11D05C0D4
:1047500026E8230F0296A11DB11D2093E205809348
:10476000E3059093E405A093E505B093E6058091F9
:10477000E7059091E805A091E905B091EA05019659
:10478000A11DB11D8093E7059093E805A093E9056D
:10479000B093EA05BF91AF919F918F913F912F9177
:1047A0000F900FBE0F901F9018952FB7F89460913F
:1047B000E3057091E4058091E5059091E6052FBF32
:1047C00008953FB7F8948091E7059091E805A0918E
:1047D000E905B091EA0526B5A89B05C02F3F19F061
:1047E0000196A11DB11D3FBF6627782F892F9A2FF3
:1047F000620F711D811D911D42E0660F771F881F9A
:10480000991F4A95D1F70895CF92DF92EF92FF92C8
:10481000CF93DF936B017C010E94E123EB01C11474
:10482000D104E104F10489F00E94F2290E94E123FD
:104830006C1B7D0B683E734090F381E0C81AD10871
:10484000E108F108C851DC4FEACFDF91CF91FF902A
:10485000EF90DF90CF900895789484B5826084BD06
:1048600084B5816084BD85B5826085BD85B5816074
:1048700085BDEEE6F0E0808181608083E1E8F0E0D4
:104880001082808182608083808181608083E0E803
:10489000F0E0808181608083E1EBF0E080818460E2
:1048A0008083E0EBF0E0808181608083EAE7F0E0E4
:1048B0008081846080838081826080838081816048
:1048C00080838081806880831092C10008958093E6
:1048D000500108958E3008F08E508770209150015D
:1048E00090E4299F90011124822B80937C00809179
:1048F0007A00806480937A0080917A0086FDFCCFF4
:10490000809178002091790090E0922B08951F9378
:10491000CF93DF93182FEB0161E00E940F252097C2
:1049200011F460E004C0CF3FD10539F461E0812F7C
:10493000DF91CF911F910C944825E12FF0E0E359CE
:10494000FD4FE491E330F9F048F4E130B9F0E230A2
:10495000A1F584B5806284BDC8BD34C0E730E9F0FC
:10496000E83019F1E43049F580918000806280934D
:104970008000D0938B00C0938A0024C084B58068E7
:1049800084BDC7BD1FC08091800080688093800077
:10499000D0938900C093880015C08091B0008068D2
:1049A0008093B000C093B3000DC08091B0008062CE
:1049B0008093B000C093B40005C0C038D1050CF09E
:1049C000B5CFAFCFDF91CF911F910895833081F0A4
:1049D00028F4813099F08230A1F008958730A9F051
:1049E0008830B9F08430D1F4809180008F7D03C08D
:1049F000809180008F7780938000089584B58F77B1
:104A000002C084B58F7D84BD08958091B0008F77FA
:104A100003C08091B0008F7D8093B0000895CF9344
:104A2000DF9390E0FC01EF57FD4F2491FC01EB5622
:104A3000FD4F8491882349F190E0880F991FFC0174
:104A4000ED54FD4FA591B49187559D4FFC01C59143
:104A5000D4919FB7611108C0F8948C91209582235E
:104A60008C93888182230AC0623051F4F8948C912F
:104A7000322F309583238C938881822B888304C0C6
:104A8000F8948C91822B8C939FBFDF91CF910895E6
:104A90000F931F93CF93DF931F92CDB7DEB7282FCD
:104AA00030E0F901E359FD4F8491F901EF57FD4FD3
:104AB0001491F901EB56FD4F04910023C9F08823AE
:104AC00021F069830E94E6246981E02FF0E0EE0F77
:104AD000FF1FE755FD4FA591B4919FB7F8948C91B6
:104AE000611103C01095812301C0812B8C939FBF5E
:104AF0000F90DF91CF911F910F9108951F920F9208
:104B00000FB60F9211242F938F939F93EF93FF93E0
:104B1000E091FB05F091FC058081E0910106F091A8
:104B2000020682FD12C09081809104068F5F8F7310
:104B300020910506821751F0E0910406F0E0E5515E
:104B4000FA4F958F8093040601C08081FF91EF9109
:104B50009F918F912F910F900FBE0F901F901895DE
:104B60001F920F920FB60F9211242F933F934F93E2
:104B70005F936F937F938F939F93AF93BF93EF93C5
:104B8000FF938BEE95E00E947026FF91EF91BF910D
:104B9000AF919F918F917F916F915F914F913F91D5
:104BA0002F910F900FBE0F901F9018958BEE95E0F0
:104BB0000E94332621E0892B09F420E0822F0895FA
:104BC0001092EE051092ED0588EE93E0A0E0B0E0C3
:104BD0008093EF059093F005A093F105B093F20553
:104BE0008BEE94E09093EC058093EB0585EC90E0E0
:104BF0009093F8058093F70584EC90E09093FA0584
:104C00008093F90580EC90E09093FC058093FB0580
:104C100081EC90E09093FE058093FD0582EC90E09E
:104C2000909300068093FF0586EC90E09093020637
:104C30008093010610920406109205061092060653
:104C400010920706089508950E942C240E9423269E
:104C50000E945A10C2E6D6E20E94E7202097E1F3B4
:104C60000E946226F9CFFC01818D228D90E0805C4C
:104C70009F4F821B910960E470E00E94122C0895FE
:104C8000FC01918D828D981731F0828DE80FF11D16
:104C9000858D90E008958FEF9FEF0895FC01918D31
:104CA000828D981761F0828DDF01A80FB11D5D968E
:104CB0008C91928D9F5F9F73928F90E008958FEFFC
:104CC0009FEF089586ED95E2892B49F080E090E012
:104CD000892B29F00E94D62581110C94000008959B
:104CE000FC01848DDF01A80FB11DA35ABF4F2C9189
:104CF000848D90E001968F739927848FA689B78958
:104D00002C93A089B1898C9180648C93938D848D30
:104D1000981306C00288F389E02D80818F7D8083FF
:104D20000895CF93DF93EC01888D8823C9F0EA8939
:104D3000FB89808185FD05C0A889B9898C9186FD94
:104D40000FC00FB607FCF5CF808185FFF2CFA88991
:104D5000B9898C9185FFEDCFCE010E947026E7CFF7
:104D6000DF91CF910895CF92DF92FF920F931F931F
:104D7000CF93DF931F92CDB7DEB76C01DC015B965A
:104D80009C915B975C968C915C97981307C05096AA
:104D9000ED91FC915197808185FD32C0F601038D24
:104DA00010E00F5F1F4F0F731127F02EF601848D57
:104DB000F81211C00FB607FCF9CFD6015096ED914D
:104DC000FC915197808185FFF1CFC60169830E94D4
:104DD00070266981EBCF838DE80FF11DE35AFF4FF9
:104DE0006083D6015B960C935B975296ED91FC9194
:104DF000539780818062808381E058968C930DC0A8
:104E0000D6015696ED91FC91579760835096ED919F
:104E1000FC91519780818064808381E090E00F90C5
:104E2000DF91CF911F910F91FF90DF90CF90089568
:104E3000BF92CF92DF92EF92FF92CF93DF93EC017C
:104E40006A017B01B22EE889F98982E080834115ED
:104E500081EE580761057105A1F060E079E08DE30E
:104E600090E0A70196010E94262C215031094109AA
:104E700051095695479537952795211580E13807B3
:104E800098F0E889F989108260E874E88EE190E092
:104E9000A70196010E94262C215031094109510990
:104EA0005695479537952795EC85FD853083EE859A
:104EB000FF852083188EEC89FD89B082EA89FB8901
:104EC000808180618083EA89FB898081886080831A
:104ED000EA89FB89808180688083EA89FB898081F7
:104EE0008F7D8083DF91CF91FF90EF90DF90CF9007
:104EF000BF90089570E09B01382BC9010895CF92AF
:104F0000DF92EF92FF920F931F93CF93DF936C0189
:104F10007A01EB01E60EF71E00E010E0CE15DF058A
:104F200061F06991D601ED91FC910190F081E02D45
:104F3000C6010995080F191FF1CFC801DF91CF9164
:104F40001F910F91FF90EF90DF90CF900895611522
:104F5000710581F0DB010D900020E9F7AD014150B2
:104F60005109461B570BDC01ED91FC910280F38146
:104F7000E02D099480E090E00895EF92FF920F9366
:104F80001F93CF93DF938C01FB01C0E0D0E06491CD
:104F90007F018FEFE81AF80A662361F0D801ED91DE
:104FA000FC910190F081E02DC8010995C80FD91F2F
:104FB000F701EDCFCE01DF91CF911F910F91FF90BF
:104FC000EF9008950C94A727DC01ED91FC910190DE
:104FD000F081E02D09940F931F93CF93DF93EC01A1
:104FE0006DE00E94E4278C016AE0CE010E94E42774
:104FF000800F911FDF91CF911F910F9108950F9313
:105000001F93CF93DF93EC010E94BD278C01CE014B
:105010000E94EB27800F911FDF91CF911F910F917D
:1050200008950F931F93CF93DF93EC010E94A7275E
:105030008C01CE010E94EB27800F911FDF91CF9151
:105040001F910F9108958F929F92AF92BF92CF922E
:10505000DF92EF92FF920F931F93CF93DF93CDB721
:10506000DEB7A1970FB6F894DEBF0FBECDBF7C01AF
:10507000C42EE52FCB01D22E19A221E02D1510F060
:105080002AE0D22E8E010F5D1F4F8D2C912CA12C6A
:10509000B12C6C2D7E2FA50194010E94262C8C2D05
:1050A000D29E80191124015011098A3014F4805DB8
:1050B00001C0895CF8018083211531054105510546
:1050C00021F0C22EE32FCA01E4CFB801C7010E942C
:1050D000A727A1960FB6F894DEBF0FBECDBFDF9114
:1050E000CF911F910F91FF90EF90DF90CF90BF90E5
:1050F000AF909F908F900895CF92DF92EF92FF92A2
:105100000F931F93CF93DF93EC016A017B0121156D
:10511000310579F4E881F9810190F081E02D642F67
:10512000DF91CF911F910F91FF90EF90DF90CF9083
:1051300009942A303105E9F477FF1AC06DE20E9424
:10514000E4278C0144275527BA014C195D096E09E3
:105150007F092AE0CE010E942328800F911FDF9152
:10516000CF911F910F91FF90EF90DF90CF90089516
:105170002AE0B701A601CE01DF91CF911F910F91D7
:10518000FF90EF90DF90CF900C9423289A01AB0111
:10519000662757FD6095762F0C947C280F931F93FC
:1051A000CF93DF93EC019A01AB01662757FD609521
:1051B000762F0E947C288C01CE010E94EB27800F65
:1051C000911FDF91CF911F910F9108952115310506
:1051D00041F4DC01ED91FC910190F081E02D642F10
:1051E00009940C9423284F925F926F927F928F9232
:1051F0009F92AF92BF92CF92DF92EF92FF920F9366
:105200001F93CF93DF93EC016A017B01B22E9A01C9
:10521000AB01C701B6010E940E2C882319F067EF7D
:1052200074E027C026013701E89477F82FEF3FEFAD
:105230004FE75FE7C301B2010E940E2C81110DC040
:105240002FEF3FEF4FE75FE7C301B2010E94582AFB
:1052500018161CF46BEF74E00CC02FEF3FEF4FE714
:105260005FE4C701B6010E94A72B1816ACF46FEFDC
:1052700074E0CE01DF91CF911F910F91FF90EF90DD
:10528000DF90CF90BF90AF909F908F907F906F9066
:105290005F904F900C94A7272FEF3FEF4FE75FEC05
:1052A000C701B6010E94582A87FDE1CF20E030E017
:1052B000A901C701B6010E94582A87FF0AC06DE202
:1052C000CE010E94E4278C01F7FAF094F7F8F094ED
:1052D00002C000E010E0A12C60E070E080E09FE3FD
:1052E000AB1441F020E030E040E251E40E945C2A3F
:1052F000A394F6CF9B01AC01C701B6010E94F4292B
:105300006B017C010E94C92A2B013C010E94F52AF5
:105310009B01AC01C701B6010E94F3296B017C011E
:105320002AE0B301A201CE010E942328080F191F11
:10533000BB2039F063E075E0CE010E94A727080F7B
:10534000191F7B2C772041F120E030E040E251E44E
:10535000C701B6010E94AB2B6B017C010E94C42ADD
:105360004B01AA2497FCA094BA2C2AE030E0B501A6
:10537000A401CE010E947C28080F191FC501B401A9
:105380000E94F72A9B01AC01C701B6010E94F329D4
:105390006B017C017A94D6CFC801DF91CF911F9128
:1053A0000F91FF90EF90DF90CF90BF90AF909F90C4
:1053B0008F907F906F905F904F9008950C94F3289A
:1053C0000F931F93CF93DF93EC010E94F3288C017E
:1053D000CE010E94EB27800F911FDF91CF911F918B
:1053E0000F91089508955058BB27AA270ED075C174
:1053F00066D130F06BD120F031F49F3F11F41EF4F0
:105400005BC10EF4E095E7FB51C1E92F77D180F342
:10541000BA17620773078407950718F071F49EF5B1
:105420008FC10EF4E0950B2EBA2FA02D0B01B90100
:1054300090010C01CA01A0011124FF27591B99F00A
:10544000593F50F4503E68F11A16F040A22F232F16
:10545000342F4427585FF3CF469537952795A79566
:10546000F0405395C9F77EF41F16BA0B620B730B0D
:10547000840BBAF09150A1F0FF0FBB1F661F771F7E
:10548000881FC2F70EC0BA0F621F731F841F48F433
:10549000879577956795B795F7959E3F08F0B3CFB9
:1054A0009395880F08F09927EE0F979587950895A3
:1054B000D9D008F481E008950CD00FC107D140F095
:1054C000FED030F021F45F3F19F0F0C0511139C126
:1054D000F3C014D198F39923C9F35523B1F3951B65
:1054E000550BBB27AA2762177307840738F09F5F05
:1054F0005F4F220F331F441FAA1FA9F333D00E2E74
:105500003AF0E0E830D091505040E695001CCAF7E0
:1055100029D0FE2F27D0660F771F881FBB1F2617A5
:1055200037074807AB07B0E809F0BB0B802DBF0178
:10553000FF2793585F4F2AF09E3F510568F0B6C091
:1055400000C15F3FECF3983EDCF386957795679555
:10555000B795F7959F5FC9F7880F911D9695879529
:1055600097F90895E1E0660F771F881FBB1F621748
:1055700073078407BA0720F0621B730B840BBA0B06
:10558000EE1F88F7E095089504D06894B111D9C052
:105590000895BCD088F09F5790F0B92F9927B75144
:1055A000A0F0D1F0660F771F881F991F1AF0BA95E7
:1055B000C9F712C0B13081F0C3D0B1E00895C0C0C6
:1055C000672F782F8827B85F39F0B93FCCF38695DD
:1055D00077956795B395D9F73EF49095809570953A
:1055E00061957F4F8F4F9F4F0895E89409C097FBB7
:1055F0003EF490958095709561957F4F8F4F9F4FAA
:105600009923A9F0F92F96E9BB279395F6958795ED
:1056100077956795B795F111F8CFFAF4BB0F11F4B0
:1056200060FF1BC06F5F7F4F8F4F9F4F16C0882357
:1056300011F096E911C0772321F09EE8872F762F8D
:1056400005C0662371F096E8862F70E060E02AF0CE
:105650009A95660F771F881FDAF7880F96958795BA
:1056600097F90895990F0008550FAA0BE0E8FEEF8F
:1056700016161706E807F907C0F012161306E40716
:10568000F50798F0621B730B840B950B39F40A260F
:1056900061F0232B242B252B21F408950A2609F4ED
:1056A000A140A6958FEF811D811D089597F99F67F1
:1056B00080E870E060E008959FEF80EC089500249A
:1056C0000A941616170618060906089500240A9467
:1056D00012161306140605060895092E0394000CED
:1056E00011F4882352F0BB0F40F4BF2B11F460FF7C
:1056F00004C06F5F7F4F8F4F9F4F089557FD9058A5
:10570000440F551F59F05F3F71F04795880F97FB85
:10571000991F61F09F3F79F087950895121613063F
:105720001406551FF2CF4695F1DF08C0161617066E
:105730001806991FF1CF86957105610508940895A3
:10574000E894BB2766277727CB0197F908958ADF6E
:1057500008F48FEF08950BD0C0CFB1DF28F0B6DF8B
:1057600018F0952309F0A2CFA7CF1124EACFC6DF06
:10577000A0F3959FD1F3950F50E0551F629FF00164
:10578000729FBB27F00DB11D639FAA27F00DB11DBD
:10579000AA1F649F6627B00DA11D661F829F222746
:1057A000B00DA11D621F739FB00DA11D621F839FCD
:1057B000A00D611D221F749F3327A00D611D231FA3
:1057C000849F600D211D822F762F6A2F11249F57F1
:1057D00050408AF0E1F088234AF0EE0FFF1FBB1F14
:1057E000661F771F881F91505040A9F79E3F5105B3
:1057F00070F05CCFA6CF5F3FECF3983EDCF386956C
:1058000077956795B795F795E7959F5FC1F7FE2B5D
:10581000880F911D9695879597F9089523DF880B3A
:10582000990B089597FB072E16F4009407D077FD87
:1058300009D00E94482C07FC05D03EF49095819534
:105840009F4F0895709561957F4F0895A1E21A2E9C
:10585000AA1BBB1BFD010DC0AA1FBB1FEE1FFF1F14
:10586000A217B307E407F50720F0A21BB30BE40B64
:10587000F50B661F771F881F991F1A9469F76095AB
:105880007095809590959B01AC01BD01CF01089565
:10589000AA1BBB1B51E107C0AA1FBB1FA617B70756
:1058A00010F0A61BB70B881F991F5A95A9F7809572
:1058B0009095BC01CD010895EE0FFF1F0590F49166
:1058C000E02D0994F999FECF92BD81BDF89A9927F0
:1058D00080B50895262FF999FECF1FBA92BD81BDDC
:1058E00020BD0FB6F894FA9AF99A0FBE0196089562
:0458F000F894FFCF5A
:1058F40000008C0680000100000001CDCC4C40FF6C
:10590400FF00006041FFFF0000C64200D084451440
:1059140000013333734060EA00000097490100003E
:10592400803FCDCC8440C409000032000000D00781
:10593400000005000000003F333383400A000000EC
:10594400013C00756E646F636B65642000756E6B5B
:105954006E6F776E200025005F6368617267696E01
:1059640067002063656C6C733A005F005F69646C68
:10597400653A005F73683A0041005F7343563A002A
:105984005F7349563A005F73563A005F70776D3A19
:10599400005F616D70733A005F6D41683A005F6C3F
:1059A400563A005F63433A005F62503A005F6552C3
:1059B4003A0068696768204348415247494E472086
:1059C40063656C6C00686967682063757272656EE4
:1059D40074003C77616C6C706F7765723E00626135
:1059E400747420736166657479207377697463686D
:1059F400204F4E0062617474506C757350696E2050
:105A04004C4F5720286E6F20666C6F7729006261B7
:105A14007474506C757350696E2048494748202847
:105A2400666C6F7729003C706F7765725F65727280
:105A34006F722000303E002C003C73687574646FF4
:105A4400776E3E0077726974696E67206572726F53
:105A54007220746F20656570726F6D003C7265739F
:105A640065743E003C636861726765643E003C6433
:105A74006F636B65643E006175746F206368617267
:105A84006765204F4E003C756E646F636B65643EC2
:105A9400006175746F20636861726765204F4646C4
:105AA400000A6D6178206368617267652074696DAE
:105AB400650A000A707265636F6E646974696F6E5B
:105AC400696E670A000A7A65726F2063757272657F
:105AD4006E740A006E65772063757272656E742049
:105AE40063616C3A2000626174742073616665744A
:105AF4007920737769746368204F46460064616E49
:105B04006765726F75736C79206C6F772063656C51
:105B14006C003C7265646F636B3E003C6869676847
:105B24005F63757272656E743E007368756E74316E
:105B3400204F4646007368756E7431204F4E0073D3
:105B440068756E7432204F4646007368756E743201
:105B5400204F4E007368756E7433204F46460073B1
:105B640068756E7433204F4E007368756E747320BD
:105B7400616C6C206F666600766F6C74732050578E
:105B84004D203000766F6C74732050574D203130A7
:105B94003000766F6C74732050574D2032303000D3
:105BA400766F6C74732050574D2032353500616424
:105BB4006A566F6C7473204F46460061646A566F70
:105BC4006C7473204F4E0061646A416D7073204F92
:105BD40046460061646A416D7073204F4E007461E3
:105BE4007267657420416D7073202B302E30350040
:105BF40074617267657420416D7073202D302E308E
:105C0400350074617267657420766F6C7473202B31
:105C1400302E30320074617267657420766F6C7454
:105C240073202D302E30323A200070777250574D49
:105C3400202B31300070777250574D202D313000B9
:105C440070777250574D202B310070777250574D3A
:105C5400202D310066756C6C6175746F204F46465B
:105C64000066756C6C6175746F204F4E003C6964FE
:105C74003A3A6F63756C7573506F7765723E003C8A
:105C84006D416843617061636974793A20003C6DC9
:105C940041683A20003C656570726F6D5F657261A2
:105CA4007365643E003C77726974696E675F746FF4
:105CB4005F656570726F6D3E003C646F636B566F19
:105CC4006C746167653A20003C5348555454494EFE
:105CD40047444F574E3E0000000000B3267F273351
:105CE400264E26402691266E616E00696E66006F10
:065CF4007666002E0000A0
:00000001FF
